:100000000C94B1170C94D9170C94D9170C94FA21AD
:100010000C94FA210C94FA210C94D9170C94D9174A
:100020000C94D9170C94D9170C94D9170C94D91790
:100030000C94D9170C94D9170C94D9170C94D91780
:100040000C94CA290C94D9170C94702C0C94A22CE3
:100050000C94D9170C94D9170C94D9170C94D91760
:100060000C94D9170C94D917FFE0FFD1AFFF32FFE2
:10007000D0FFFEFFE0FFD1AEFFD0FFFEFFE0FFD1DB
:100080001000FFFEFFD0FFE0FFC1FFD1AED580A87A
:100090003FD300408D142000A1C8DA1281CFD9F1DE
:1000A000DB402EA4A6AFFFD0FFFE000D12FEFC0821
:1000B00001B2036F20FFFE0BFE08FE0000000300EC
:1000C0000101080803010080808080808000800397
:1000D0000202040106A0A006070706000028287CEB
:1000E00028F85050050A0A0600FF2070A8A07028C2
:1000F00028A87020080808090000649468081016F1
:100100002926060808080100609090609488986489
:100110000102020200068080030A0A0400FE204059
:100120004080808080404020030A0A0401FE804015
:100130004020202020404080030303040005A0400D
:10014000A00505050600012020F820200203030376
:1001500000FE404080030101040003E001010103AF
:100160000100800308080300002020404040408038
:1001700080050808060000708888888888887002D2
:10018000080806010040C0404040404040050808C3
:1001900006000070880808304080F805080806004E
:1001A00000708808300808887005080806000010EC
:1001B00030505090F81010050808060000784040B4
:1001C0007008088870050808060000708880F088AC
:1001D000888870050808060000F8081020204040B4
:1001E00040050808060000708888708888887005B7
:1001F000080806000070888888780888700106065C
:100200000301008000000000800208080300FE4097
:1002100000000000404080030505060101204080E9
:100220004020040303050002F000F0030505060169
:1002300001804020408004080806010060901020E2
:10024000404000400A09120B00FF1F0020804D4073
:100250009240A240A4809B0040003E00070808078F
:10026000000010102828447C82820508080701003D
:10027000F08888F0888888F00608080801007884EB
:10028000808080808478060808080100F0888484D3
:10029000848488F0050808070100F88080F88080D1
:1002A00080F8050808060100F88080F080808080D2
:1002B000060808080100788480808C84847C060805
:1002C00008080100848484FC848484840108080371
:1002D0000100808080808080808004080805000004
:1002E0001010101010109060050808070100889089
:1002F000A0E0909088880408080601008080808033
:10030000808080F007080809010082C6C6AAAA9268
:100310009292060808080100C4C4A4A494948C8C8A
:100320000608080801007884848484848478050899
:1003300008070100F08888F080808080070909089C
:1003400001FF7884848484948C7C0205080807016A
:1003500000F08888F0888888880508080701007000
:1003600088807008888870050808050000F820203B
:10037000202020202006080808010084848484842A
:1003800084847807080807000082824444442828AF
:10039000100908100900008880888049004900552C
:1003A000002200220022000508080701008888506A
:1003B00020505088880708080700008244442828F5
:1003C000101010050808070100F8081020204080D0
:1003D000F8020A0A0301FEC080808080808080804D
:1003E000C0030808030000808040404040202002F5
:1003F0000A0A0300FEC04040404040404040C00563
:10040000050506000320205050880601010600FE65
:10041000FC0202020300078040050606050000E01A
:1004200010709090680508080600008080B0C888A9
:1004300088C8B004060605000060908080906005C2
:100440000808060000080868988888986804060666
:100450000500006090F080906004080804000030FF
:1004600040E040404040400508080600FE6898888B
:1004700088986808700508080600008080B0C88861
:1004800088888801080802000080008080808080C1
:1004900080020A0A02FFFE400040404040404040C7
:1004A00080040808050000808090A0C0A090900102
:1004B0000808020000808080808080808007060617
:1004C000080000EC9292929292050606060000B097
:1004D000C88888888805060606000070888888888D
:1004E000700508080600FEB0C88888C8B08080057E
:1004F00008080600FE6898888898680808030606B9
:10050000040000A0C0808080800406060500006012
:1005100090601090600308080400004040E04040F4
:100520004040600406060500009090909090700591
:10053000060606000088885050202007060608009E
:100540000092925454282805060606000088502080
:1005500050888805080805FFFE4848505030202084
:10056000C0040606050000F010204080F0030A0ACF
:100570000300FE20404040804040404020010A0AE5
:100580000301FE80808080808080808080030A0A52
:100590000300FE8040404020404040408006020270
:1005A0000700036498FFFFFFFFFFFFFFFFFFFFFF50
:1005B000FFFFFFFFFFFFFFFFFFFFFFFFFFFFFFFF4B
:1005C000FFFFFFFFFFFF0000000300010108080319
:1005D00001FE80008080808080800508080601FF81
:1005E0001070A8A0A0A870400508080600003048B8
:1005F00040E0404048B0040606050001906090903D
:10060000609005080806000088888850F820F820C7
:10061000010A0A0301FE80808080000080808080C3
:10062000050A0A0600FE7088C07098C870188870A5
:10063000030101030007A007070709010038449AD6
:10064000A29A4438030505040003E020A000E00559
:1006500005050600002850A05028050303070102E5
:10066000F80808030101040003E007070709010077
:100670003844BAB2AA4438030101030007E0040475
:100680000404000460909060050707060000202025
:10069000F8202000F803040403000460A040E003F5
:1006A0000404030004E04020C002020203000740EB
:1006B000800408080500FE9090909090F0808006DD
:1006C0000A0A0600FE7CE8E8E868282828282802AC
:1006D0000101030003C00202020300FE40C0020445
:1006E0000403000440C04040030505040003E0A0EB
:1006F000E000E0050505060000A0502850A009080C
:10070000100900004400C400480048001100130014
:100710002780210008080809000044C44848131530
:100720002227090810090000E00044002400C80046
:1007300009001300178021000408080601FE2000AC
:10074000202040809060070B0B0700002010001055
:10075000102828447C8282070B0B07000008100039
:1007600010102828447C8282070B0B0700001028F9
:100770000010102828447C8282070B0B070000140D
:10078000280010102828447C8282070A0A070000EB
:10079000280010102828447C8282070B0B070000D9
:1007A00010281010102828447C82820908100A00A2
:1007B000001F80180028002F804800780088008FD4
:1007C00080060A0A0801FE78848080808084781080
:1007D00030050B0B070100402000F88080F8808076
:1007E00080F8050B0B070100102000F88080F880CE
:1007F0008080F8050B0B070100205000F88080F87E
:10080000808080F8050A0A0701005000F88080F80F
:10081000808080F8020B0B030000804000404040C5
:100820004040404040020B0B0301004080008080AC
:10083000808080808080030B0B03000040A000407C
:1008400040404040404040030A0A030000A00040EE
:1008500040404040404040070808080000784442BB
:10086000F242424478060B0B080100285000C4C431
:10087000A4A494948C8C060B0B0801002010007823
:1008800084848484848478060B0B0801000810009B
:100890007884848484848478060B0B0801002050BB
:1008A000007884848484848478060B0B08010028F3
:1008B00050007884848484848478060A0A080100BD
:1008C00048007884848484848478050505060001C2
:1008D0008850205088060A0A0801FF04788C9494F6
:1008E000A4A4C47880060B0B0801002010008484A7
:1008F000848484848478060B0B080100081000842B
:1009000084848484848478060B0B080100205000C2
:100910008484848484848478060A0A080100480058
:100920008484848484848478070B0B070000081077
:100930000082444428281010100508080701008090
:1009400080F08888F080800408080500006090909E
:10095000A0909090A0050909050000402000E0103B
:1009600070909068050909050000204000E01070B3
:10097000909068050909050000205000E010709073
:10098000906805090905000050A000E010709090E3
:10099000680508080500005000E010709090680598
:1009A0000909050000205020E010709090680706AB
:1009B00006080000EC127E90926C0408080500FE08
:1009C000609080809060206004090905000040204C
:1009D000006090F08090600409090500002040004C
:1009E0006090F080906004090905000040A000605C
:1009F00090F0809060040808050000A0006090F06E
:100A000080906002090902FF0080400040404040A1
:100A10004040020909020000408000808080808000
:100A20008003090902FF0040A000404040404040D0
:100A300003080802FF00A000404040404040050974
:100A40000906000040789078888888887004090931
:100A500005000050A000E0909090909005090906D4
:100A60000000402000708888888870050909060009
:100A70000010200070888888887005090906000029
:100A800020500070888888887005090906000028B1
:100A9000500070888888887005080806000050009B
:100AA0007088888888700505050600012000F80018
:100AB0002007060606FF003A4C546444B8040909AE
:100AC0000500004020009090909090700409090566
:100AD000000010200090909090907004090905008B
:100AE0000040A000909090909070040808050000CD
:100AF000A000909090909070050B0B05FFFE0810E1
:100B00000048485050302020C0050A0A0600FE80E8
:100B100080B0C88888C8B08080050A0A05FFFE50EA
:100B20000048485050302020C0002F2CF0F614040C
:100B3000DC0B9020FFF81BF719F8000000070000FD
:100B40000417170902003070707070707070706058
:100B500060606060606060400070F0F0E0080A0A69
:100B60000E030DE3C7C7C7C7C3C3C3C3C20E122456
:100B70000F0102011803180310023006303FFC0475
:100B8000600C600C600C4008C0FFF81880118031C8
:100B9000803180310023000C19320F01FD06000660
:100BA0000006001FC03FF0666066006600660076C3
:100BB000003E001F8007C007E00670063006308642
:100BC00030C630E660FFC07F8006000600060014D5
:100BD000143C1601FF1E00C0630180430380C183E3
:100BE00000C18600C18C00C19C0061180063300008
:100BF0003C73C0006C6000C86001983003983003FB
:100C000018300618300E08201C0C601807803000C1
:100C10000013164215020003C00004E00008600043
:100C200018600018600018600018C0001D80000FD8
:100C300000000C00001C3FE03E0E8077060063863B
:100C400000C18600C1C600C0EC00C07C00C03C00F2
:100C5000601E00302FC01FC380030A0A08030DE086
:100C6000C0C0C0C0C0C0C0C0C0071E1E0A02FB0278
:100C70000C1818303060606060C0C0C0C0C0C0C018
:100C8000C0C0C0E0606060703038180C02071E1EE3
:100C90000A01FB80603038181C0C0C0C0E0606068E
:100CA000060606060606060C0C0C0C1818303060FA
:100CB000800C0D1A0E010B0600060086006630F24D
:100CC000F01B8006001B8072F0E63006200600064E
:100CD000000C0B160D0103060006000600060006B8
:100CE00000FFF006000600060006000600040808E3
:100CF0000702FB70F03030302040C00901020B01C8
:100D000008FF8004040407020070F0F0E00D1E3CB0
:100D10000F01FB0018003800300030007000600048
:100D20006000E000C001C001800180038003000773
:100D300000060006000E000C000C001C0018003815
:100D40000030003000700060006000E000C0000D66
:100D500013260F0100078018C0206060304030402B
:100D600038C018C018C018C018C018C018C018C0A3
:100D70001060106030302018400F800B13260F02D7
:100D80000002001E007E0086000600060006000627
:100D90000006000600060006000600060006000623
:100DA0000006000F007FE00B13260F02000F8030BB
:100DB000C06060606060600060006000C000C001F2
:100DC000800300070006000C00180030207020E0AF
:100DD00020FFE00B13260F02001F00718060C0E0AF
:100DE000C000C000C0018003000F0003C000C000AD
:100DF000E0006000600060006080C0C1807F000C87
:100E000013260F0100004001C003C003C006C00C40
:100E1000C00CC018C030C030C060C0E0C0FFF000DF
:100E2000C000C000C000C000C007F00B13260F02B6
:100E3000003FE02000200060006000600060007F54
:100E40000061C000C00060006000600060006000E1
:100E50004080C0C1803F000C14280F020000C00772
:100E6000000E0018003000700060006000CF80F0BD
:100E7000E0E060C070C030C030C030603060202022
:100E80006030400F800C13260F0200FFF08060805E
:100E90006000E000C000C001800180030003000783
:100EA00000060006000C000C001C00180038003082
:100EB000000C13260F02001F8030C06060E060E06D
:100EC00060E060F8C07F801F801FC031E06070C0AC
:100ED00070C030C030C020602070401F800C1428CB
:100EE0000F02FF0F8031C020E04060C070C030C0F2
:100EF00030C030C030607030B01F30006000600023
:100F00006000C0018007001E003000040F0F0702C0
:100F10000070F0F0600000000000000070F0F0E0F1
:100F20000414140702FB70F0F060000000000000E1
:100F3000000070F03030302040C00C0A140E010464
:100F4000003000F007C03E00F800F0007E000F8087
:100F500001F000700C060C0E0106FFF0000000000E
:100F600000000000FFF00C0A140E01046000F800FD
:100F70001F0007E000F001F007C03E00F000C000D5
:100F80000A172E0E02001F00638041C0C0C0C0C0FF
:100F900080C000C0018001800300030006000E0035
:100FA0000C000C000C000C00000000000E001E00E5
:100FB0001E001C0018194B1A01FB003F8001C0E005
:100FC0000200380C001C18000C103C8E2043866078
:100FD0008187418183C10183C30183C30183C3012D
:100FE00083C30183C30183C30182E181866183845A
:100FF00070C5C83078F03800001C00040F001C03D6
:10100000C070007F8013143C13000000400000E01B
:101010000000E00001E00001F00001B0000330003A
:10102000033800031800061C00061C00060C000F05
:10103000FE000C0600080600180700180300100345
:1010400000300380FE0FE00E14281101003FC0F0B5
:101050007030383018301830183018303030E03FE9
:10106000E030703038301C300C300C300C300C302C
:10107000183030FFC00E142811010003F80C1C10AA
:10108000083000600060004000C000C000C000C028
:1010900000C000C000C00060006000700038041C88
:1010A0001807E011143C1301003FE000F038003055
:1010B0000C003006003003003003003003803001A4
:1010C000803001803001803001803001803001802B
:1010D000300300300300300300300600300C0030D5
:1010E0003800FFE0000D1428100100FFF030103030
:1010F000103010300030003000300030003FE03061
:10110000403000300030003000300030083008300F
:1011100018FFF80C14280F0100FFF03010301030C9
:1011200010300030003000300030003FC0308030E0
:10113000003000300030003000300030003000FE61
:101140000012143C13010001FE00060F000800000D
:10115000100000200000600000400000C00000C03F
:101160000000C00000C00000C01FC0C00700C003D6
:10117000006003006003003003001803000C03004C
:1011800003FC0013143C150100FC07E03001803023
:1011900001803001803001803001803001803001D9
:1011A000803001803FFF803001803001803001803D
:1011B000300180300180300180300180300180308A
:1011C0000180FC07E00614140A0200FC30303030C5
:1011D0003030303030303030303030303030FC0B68
:1011E00019320AFDFB0FE0018001800180018001BE
:1011F00080018001800180018001800180018001E7
:101200008001800180018001800180018001000156
:101210000003006200FC0011143C130100FC7F007D
:1012200030180030300030600030E00031C0003154
:1012300080003300003600003E000036000037001A
:101240000033800031C00030E000307000307800A2
:10125000303C00301E00FC0F800D14280F0100FCF4
:1012600000300030003000300030003000300030FE
:1012700000300030003000300030003000300030EE
:101280000830083018FFF818143C1A0100F8003E26
:101290003C00383C00783E00783600D83600D8371D
:1012A000009833019833819831831831C31831C6BF
:1012B0001830C61830E618306C18307C18303818E2
:1012C000303818303818FC10FF13143C150100F0AA
:1012D00007E03801803C01803C01803E01803701FD
:1012E0008033818033818031C18030E18030618002
:1012F000307180303980301D80300D80300F80306B
:101300000780300380300380FC018011143C1301FE
:101310000003F0000C1800100C0030060020030041
:10132000600300400380C00180C00180C00180C014
:101330000180C00180C00180E00100600300600204
:10134000003006003804000C180007E0000F1428D5
:101350001101003FE0F038301C300E30063006300E
:10136000063006300C300C343833E03000300030BA
:10137000003000300030003000FE0013194B130124
:10138000FB03F0000C1800100C00300600200300D6
:10139000600300400380C00180C00180C00180C0A4
:1013A0000180C00180C00180E00100600300600393
:1013B000003006001804000C180007F00000700050
:1013C000001800000E200007C000018012143C121B
:1013D00001003FC000F07000301800300C00300CED
:1013E00000300C00300C003018003070003FE0007E
:1013F0003FC00031C00030E000307000307000307D
:101400003800303C00301C00300F00FC0FC00C14C2
:10141000280F02000FE030E04040C000C000E000B4
:10142000F8007E007F001FC007E001F000F00070B0
:10143000003000308020C060E0C07F00101428120F
:101440000100FFFF81838181818101800180018012
:101450000180018001800180018001800180018084
:1014600001800180018001800FF013143C15010000
:10147000FC07E03001803001803001803001803095
:1014800001803001803001803001803001803001E6
:1014900080300180300180300180300180300100D7
:1014A0001803001C06000E0C0003F00014143C1579
:1014B0000000FE03F03800C01800801C01800C0101
:1014C000800E03000E030006030007060007060057
:1014D000030600038C00018C0001CC0001D8000041
:1014E000D80000F80000F0000070000060001B143D
:1014F000501B0000FE040FE038040300180E030028
:10150000180E03001C0F03001C1B02000C1B06001E
:101510000C1B86000C3186000E3186000E31C40093
:101520000660CC000660CC000760EC0007C06C00D1
:1015300003C0780003C078000380380003803800BF
:101540000300300013143C1400007F1FC03C070050
:101550001C06000E0600070C00071C000398000183
:10156000F00001F00000E00000F00001F00001B820
:1015700000031C00070C00060E000C07001C038073
:101580003803C0FF0FE012143C130000F01FC038F6
:1015900007001C06000C0C000E0C000718000718B2
:1015A0000003300003B00001E00001E00000C000D3
:1015B00000C00000C00000C00000C00000C000006B
:1015C000C00000C00007F8000E14281101007FFCC5
:1015D000601C40384078007000E000E001C003C0AB
:1015E0000380070007000E001E001C0038003804AE
:1015F0007004F00CFFFC071E1E0A02FBFEC0C0C0F8
:10160000C0C0C0C0C0C0C0C0C0C0C0C0C0C0C0C0DA
:10161000C0C0C0C0C0C0C0C0C0FE0D1E3C0F01FB9A
:10162000C000C00060006000700030003000180092
:1016300018001C000C000C000E0006000600030041
:10164000030003800180018000C000C000C0006072
:10165000006000700030003000180018071E1E0ADD
:1016600001FBFE0606060606060606060606060632
:10167000060606060606060606060606060606FE12
:101680000C0F1E100209020006000F000F001B00C5
:101690001B80118031C031C060C060E06060C070EC
:1016A000C03080200D01020F01FDFFF80707070A77
:1016B000001060F038180C04020D0F1E0F01000F0F
:1016C000C030E070606060006000600FE03FE07E6E
:1016D00060F060E060C060C06041E03E780F1830AC
:1016E0001000003000F000300030003000300030DA
:1016F000003000300030F031F8361C3C0C380E3031
:101700000630063006300630063004300C30081C37
:101710001007E00C0F1E0E010007E018602020608B
:10172000004000C000C000C000C000C000C0006099
:1017300000702038701F800F183011010000180051
:101740007800180018001800180018001800180772
:10175000F81838201860184018C018C018C018C0F1
:1017600018C018C0186018703838DE0F180D0F1E1A
:101770000F010007C01860203060184018C018FF23
:10178000F0C000C000C000E0006000700838300FFA
:10179000C00B18300A010003E004C018001000302C
:1017A000003000300030003000FF003200300030E8
:1017B00000300030003000300030003000300030A9
:1017C0000030003000FE000F172E1001F8078618B9
:1017D000FC20606030603060306030706038401FE6
:1017E00080080010003C003FE00FF83FFC707CE0F8
:1017F0000CC00CC008601070201FC01018301201FF
:10180000001000F0003000300030003000300030B8
:1018100000300030703188360C380C380C300C3009
:101820000C300C300C300C300C300C300C300CFC0C
:101830003F06151509010030707060000030F0306F
:101840003030303030303030303030FC091D3A0824
:10185000FCF8018003800380030000000000018089
:10186000078001800180018001800180018001806A
:101870000180018001800180018001800180018060
:1018800001800100030002007C00F8000F183010F6
:1018900001001000F0003000300030003000300057
:1018A0003000300030FC307030E0318033003600E2
:1018B0003E0036003700338031C030E03070307881
:1018C000FC3E06181809010010F03030303030307E
:1018D000303030303030303030303030303030FC3C
:1018E000180F2D1A0100F0F07833198C341A0C38C7
:1018F0001C0C381C0C30180C30180C30180C30181C
:101900000C30180C30180C30180C30180C30180C27
:10191000FC7E3F100F1E1201007070B188360C382B
:101920000C380C300C300C300C300C300C300C30CF
:101930000C300C300CFC3F0E0F1E10010007C018BD
:101940007020386018401CC00CC00CC00CC00CC00B
:101950000CE0086018701038200FC00F172E11010E
:10196000F870F0B318341C380C300E3006300630E6
:1019700006300630063004300C30083C1037E030BA
:1019800000300030003000300030003000FE000E2B
:10199000172E1001F807901870203060304030C0CA
:1019A00030C030C030C030C030C0306030607030C7
:1019B000B01F300030003000300030003000300008
:1019C0003001FC0B0F1E0D010031E0F3E034403814
:1019D000403800300030003000300030003000303F
:1019E0000030003000FE00090F1E0C02003F0043D3
:1019F00000C100C000E000F8007E003F000F80033F
:101A000080018081808100C300FC000A14280B0142
:101A10000010003000300030003000FFC0310030D6
:101A20000030003000300030003000300030003036
:101A3000003000300030801F400F0F1E11010030B9
:101A400018F0783018301830183018301830183036
:101A500018301830183018303818DE0F180F0F1ED5
:101A6000100000FC3E380C380818181C180C100C1C
:101A7000300E30062007600740034003C00180019C
:101A800000160F2D170000FC107C30181838381085
:101A9000183830183C301C6C300C6E200C4E600C2A
:101AA000C6600EC7400683400783C00783C003019A
:101AB00080020100100F1E100000FE3F3C1C1C1095
:101AC0000E30066007C003C001C003C006E00C7002
:101AD0000C381818381CFC3F10172E10FFF87E1F0A
:101AE0001C061C040C0C0E0C0E080618071803101C
:101AF000033003B001A001E001E000C000C000809D
:101B00000180018003007E007C00F8000C0F1E0E97
:101B100001007FF0406040E001C0018003800700C9
:101B200006000E001C001C00381070107030FFF012
:101B3000081E1E0B02FB03060C08181818181C0CB4
:101B40000C0C0C1830F81C0C0C0C0C1C1818181869
:101B5000180C06030220200703FAC0C0C0C0C0C092
:101B6000C0C0C0C0C0C0C0C0C0C0C0C0C0C0C0C075
:101B7000C0C0C0C0C0C0C0C0C0C0081E1E0B01FB9A
:101B8000C0603018181818183830303030381F0C32
:101B900018303030303818181818103060C00E0661
:101BA0000C1001071C083E0C7F8847F083F080E092
:101BB000FFFFFFFFFFFFFFFFFFFFFFFFFFFFFFFF35
:101BC000FFFFFFFFFFFFFFFFFFFFFFFFFFFFFFFF25
:101BD000FF0000000700000418180902F770F0F079
:101BE000E000002060606060606060606070707045
:101BF00070707070400C14280F02FF06000600067B
:101C0000000FE036E066606600C600C600C600C68B
:101C100000C600C600E62076303FC01F80060006E2
:101C20000006000D13260F010007E00870103010A9
:101C30002030203000300030003000FF0030003015
:101C400000300030003008201860307FF083F00B47
:101C50000A140F0204C0607FC031C060C060C06061
:101C6000C071C03F80404080201013260FFF00F05D
:101C70003F381C1C181C380E300670076003C00368
:101C8000C0018001803FFC01800180018001800152
:101C90008001800FF00220200703FAC0C0C0C0C03E
:101CA000C0C0C0C0C0C0C0C0C080000040C0C0C074
:101CB000C0C0C0C0C0C0C0C0C0C0C00B162C0F0286
:101CC000001F8031C060806000700078003E006FAF
:101CD00080C7C0C1E0C0E0E060F0607C603FC00F42
:101CE0008003C001C040C040C060803F00090408BC
:101CF0000D02116180E380E380C30015143C1801DC
:101D00000001FC000603001800C0300060307C6059
:101D1000618630630030C20018C60018C60018C6BD
:101D20000018C60018C7001863003061C63030F8CC
:101D3000603000601800C006030001FC00070A0ABA
:101D400008010938CC8C1C6CCCDCEE00FE0C0E1C9F
:101D5000100100061004300860186030C071C0E344
:101D600080E38071C030C018600860043006100D38
:101D7000060C0F0103FFF8001800180018001800E7
:101D8000180901020B0108FF800A0B160B010B1E3C
:101D90000061007E80934097409C4094409240694F
:101DA0008021001E000A0102100313FFC00707076D
:101DB0000B020C3C6EC6C6C6EC780C0E1C0D010264
:101DC00006000600060006000600FFF006000600FA
:101DD00006000600040000000000FFE0080B0B0AEC
:101DE000010A3E63C30306060C183261FF090C1892
:101DF0000B00091F0033806180018003000F000188
:101E000080018001800180C3003E000707070A03AC
:101E1000100C1E18303060C00F172E1101F830085A
:101E2000F038301830183018301830183018301892
:101E30003018383838783FF837DE339830003000C3
:101E40003000300038003800380030000F183012F1
:101E500001FC0FFE30FC60D840D8C0D8C0D8C0D834
:101E6000C0D8E0D870D838D80FD800D800D800D85B
:101E700000D800D800D800D800D800D800D800D8A2
:101E800003FE03040405010960E0E0C0050707073D
:101E900001F9302030781830E0080B0B0B020A18DB
:101EA000F81818181818181818FF070A0A0901094D
:101EB000386CC6C6C6C66C3800FE0C0E1C1002007C
:101EC00082004100618030C038E01C600C701C70E2
:101ED0001E6038E030C0618041008200101326137C
:101EE00002003006F00E300C3018303830303060E0
:101EF00030E030C0CD82018E031E061606260C4649
:101F0000187F18863006601F0F1326120200300655
:101F1000F00C3008301830303030306030C030C015
:101F2000CD80011C0366064604060C0C18181830F8
:101F3000306260FE1113391301003C0300460600B5
:101F40000604001C0C000618000610000630008E67
:101F5000600078600000C100018700018F00030B62
:101F6000000213000623000C3F800C4300180300FE
:101F7000300F800A18300D02F70E001E001E001CE4
:101F8000000000000000000C000C000C000C001C05
:101F90000018003000300060006000C000C040C089
:101FA000C0C0C0E08061803E00131B5113000006DA
:101FB00000000F000007800001C00000600000105A
:101FC0000000000000400000E00000E00001E00030
:101FD00001F00001B00003300003380003180006D0
:101FE0001C00061C00060C000FFE000C0600080674
:101FF00000180700180300100300300380FE0FE0F4
:10200000131B51130000000800001E00003C0000DC
:10201000700001C00001000000000000400000E06E
:102020000000E00001E00001F00001B0000330001A
:10203000033800031800061C00061C00060C000FE5
:10204000FE000C0600080600180700180300100325
:1020500000300380FE0FE0131B5113000000E0006E
:1020600001E00001F000033800060C000C04000041
:10207000000000400000E00000E00001E00001F08E
:102080000001B000033000033800031800061C00F4
:10209000061C00060C000FFE000C060008060018C7
:1020A0000700180300100300300380FE0FE0131A2E
:1020B0004E13000003840007E60004FC000838000B
:1020C00000000000000000400000E00000E000010F
:1020D000E00001F00001B0000330000338000318F5
:1020E00000061C00061C00060C000FFE000C06007B
:1020F000080600180700180300100300300380FED4
:102100000FE013194B130000060C00060C000E1C08
:1021100000060C0000000000400000E00000E000AD
:1021200001E00001F00001B00003300003380003BB
:102130001800061C00061C00060C000FFE000C0612
:102140000008060018070018030010030030038081
:10215000FE0FE0131B5113000000E00001B000016E
:10216000300003300001B00001E00000000000403A
:102170000000E00000E00001E00001F00001B0001C
:10218000033000033800031800061C00061C00067C
:102190000C000FFE000C06000806001807001803CC
:1021A00000100300300380FE0FE017143C190000FC
:1021B00003FFFC007C04006C0400EC0400CC000174
:1021C000CC00018C00018C00038C0003FFF8070C8D
:1021D00010060C00060C000C0C000C0C001C0C0073
:1021E000180C02180C02300C06FC3FFE0F1B3611B7
:1021F00001F903F80C1C100830006000600040007A
:10220000C000C000C000C000C000C000E00060000E
:10221000700078023C0C1FF80FF00080008001E095
:1022200000E0006000C003000D1B3610010010002C
:1022300038001C000F00038000C00000FFF03010C9
:1022400030103010300030003000300030003FE0FF
:1022500030403000300030003000300030083008AE
:102260003018FFF80D1B36100100002000F001E0CF
:10227000038007000C000000FFF030103010301019
:10228000300030003000300030003FE0304030009F
:102290003000300030003000300830083018FFF8CF
:1022A0000D1B36100100030007800FC01CC03860F2
:1022B00020300000FFF030103010301030003000BF
:1022C0003000300030003FE030403000300030005F
:1022D00030003000300830083018FFF80D19321087
:1022E000010018303870387030600000FFF0301096
:1022F00030103010300030003000300030003FE04F
:1023000030403000300030003000300030083008FD
:102310003018FFF8091B360AFF006000F000780053
:102320001C000700010000001F80060006000600D8
:10233000060006000600060006000600060006006D
:1023400006000600060006000600060006001F80C4
:10235000081B1B0A0200060F1E38608000FC30308C
:10236000303030303030303030303030303030306D
:10237000FC0A1B360A00001C001E003E007300C150
:102380008080C000003F000C000C000C000C000C12
:10239000000C000C000C000C000C000C000C000CDD
:1023A000000C000C000C000C000C003F000A19325D
:1023B0000A0000C180E1C0E1C0C18000003F000C04
:1023C000000C000C000C000C000C000C000C000CAD
:1023D000000C000C000C000C000C000C000C000C9D
:1023E000000C003F0012143C1300001FF000781C8A
:1023F000001806001803001801801801801801C099
:102400001800C01800C0FF80C01800C01800C01815
:1024100000C01801801801801801801803001806F8
:1024200000181C007FF000131A4E150100038400F1
:1024300007E600047C00083800000000000000F0FF
:1024400007E03801803C01803C01803E018037017B
:102450008033818033818031C18030E18030618080
:10246000307180303980301D80300D80300F8030E9
:102470000780300380300380FC0180111B51130161
:10248000000C00001E00000F000003800000E000B0
:1024900000200000000003F0000C1800100C0030B9
:1024A0000600200300600300400380C00180C001DB
:1024B00080C00180C00180C00180C00180E00100B7
:1024C0006003006002003006003804000C180007AA
:1024D000E000111B51130100001800003C000078BF
:1024E0000000E00001800002000000000003F00096
:1024F0000C1800100C0030060020030060030040A0
:102500000380C00180C00180C00180C00180C00183
:1025100080C00180E001006003006002003006001E
:102520003804000C180007E000111B5113010001D2
:10253000C00001E00003E0000730000C1800080CA8
:102540000000000003F0000C1800100C0030060022
:10255000200300600300400380C00180C00180C0F0
:102560000180C00180C00180C00180E001006003E3
:10257000006002003006003804000C180007E0007C
:10258000111A4E13010003040007CC0008F80010D4
:10259000700000000000000003F0000C1800100C98
:1025A00000300600200300600300400380C001806B
:1025B000C00180C00180C00180C00180C00180E0F6
:1025C00001006003006002003006003804000C18AF
:1025D0000007E00011194B1301000C18000E1C003D
:1025E0000E1C000C180000000003F0000C18001076
:1025F0000C00300600200300600300400380C0018F
:1026000080C00180C00180C00180C00180C0018005
:10261000E001006003006002003006003804000C96
:10262000180007E0000B0A140D0104C06060C031FF
:10263000801B000E000E001B00318060C0C06011C6
:10264000153F1301FF03F180041F00180E00301E18
:1026500000201F00603F00403B80C07380C0E180CD
:10266000C0E180C1C180C38180C30180E701006EE9
:1026700003007C02007C06003804007C1800C7E0E0
:1026800000800000131B511501000600000F000020
:1026900007800001C000006000001000000000FC86
:1026A00007E030018030018030018030018030014E
:1026B0008030018030018030018030018030018025
:1026C00030018030018030018030018030010018FD
:1026D00003001C06000E0C0003F000131B51150133
:1026E00000000C00001E00003C0000700000C00054
:1026F000010000000000FC07E03001803001803064
:102700000180300180300180300180300180300153
:1027100080300180300180300180300180300180C4
:102720003001803001001803001C06000E0C00036D
:10273000F000131B5115010000E00000F00001F053
:1027400000039800060C00040600000000FC07E0EF
:1027500030018030018030018030018030018030D4
:1027600001803001803001803001803001803001F3
:10277000803001803001803001803001001803007A
:102780001C06000E0C0003F00013194B1501000687
:102790000C00070E00070E00060C00000000FC07EE
:1027A000E0300180300180300180300180300180D4
:1027B0003001803001803001803001803001803074
:1027C0000180300180300180300180300100180329
:1027D000001C06000E0C0003F000121B5113000039
:1027E000000C00001E00003C0000700000C0000152
:1027F0000000000000F01FC03807001C06000C0C91
:10280000000E0C0007180007180003300003B0008A
:1028100001E00001E00000C00000C00000C00000B6
:10282000C00000C00000C00000C00000C00007F8E9
:10283000000F1428110100FE003000300030003F6E
:10284000E03078301C300E3006300630063006306E
:102850000C300C343833E0300030003000FE001013
:10286000183012010001E006380818101C100C3056
:102870000C300C301C303830F031C03180318031B8
:10288000C030F0307C303E300F3007300331033140
:10289000033186F1F80D172E0F0100380038001CA7
:1028A000000E0006000300010000000FC030E070C1
:1028B000606060006000600FE03FE07E60F060E01C
:1028C00060C060C06041E03E780D172E0F0100002F
:1028D000E000E001C0018003000200040000000FDE
:1028E000C030E070606060006000600FE03FE07E3C
:1028F00060F060E060C060C06041E03E780D172E7F
:102900000F0100070007000F801DC018C0306020B5
:102910002000000FC030E070606060006000600F59
:10292000E03FE07E60F060E060C060C06041E03E9B
:10293000780D152A0F01001C103F2023C040000015
:102940000000000FC030E070606060006000600F49
:10295000E03FE07E60F060E060C060C06041E03E6B
:10296000780D152A0F01003060387030603060003B
:102970000000000FC030E070606060006000600F19
:10298000E03FE07E60F060E060C060C06041E03E3B
:10299000780D162C0F010007800D800CC00C800DE7
:1029A000800F0000000FC030E070606060006000C9
:1029B000600FE03FE07E60F060E060C060C06041BA
:1029C000E03E78130F2D1602001F8F0071B0C0601B
:1029D000E0C0E0E06080C06000C06007FFC01CC0D5
:1029E0000070C00060C000C0C000C0E000C1604016
:1029F000C270E07C1F000C162C0E01F907E0186075
:102A0000202060004000C000C000C000C000C00026
:102A1000E000701078603FC01F8002000200078055
:102A20000380018003000C000D172E0F0100180019
:102A30003C000C000600030001000180000007C0FC
:102A40001860203060184018C018FFF0C000C000A7
:102A5000C000E0006000700838300FC00D172E0F66
:102A60000100006000F000C001800180030006004A
:102A7000000007C01860203060184018C018FFF030
:102A8000C000C000C000E0006000700838300FC017
:102A90000D172E0F0100030007800F800CC0186077
:102AA00010202010000007C0186020306018401867
:102AB000C018FFF0C000C000C000E0006000700857
:102AC00038300FC00D152A0F0100183038703870DB
:102AD00030600000000007C0186020306018401807
:102AE000C018FFF0C000C000C000E0006000700827
:102AF00038300FC0071717090000E0E07030180CDD
:102B00000400187818181818181818181818181811
:102B10007E08171709010007070E0C183020003037
:102B2000F0303030303030303030303030FC091759
:102B30002E0900001C001C003E0077006300C180CD
:102B40008080000018007800180018001800180095
:102B500018001800180018001800180018001800B5
:102B60007E000A152A090000C180C180E3C0C1802F
:102B70000000000018007800180018001800180065
:102B80001800180018001800180018001800180085
:102B90007E000E172E1001000C003E1803F003C03B
:102BA0001EE030600070003807981878203C601CE8
:102BB000400CC00CC00CC00CC00CC008E018601069
:102BC000703038600F8010152A12010007080F902E
:102BD00018E01000000000007070B188360C380C4E
:102BE000380C300C300C300C300C300C300C300CFD
:102BF000300C300CFC3F0E172E1001001C001C0086
:102C00000E000600030001800080000007C018705D
:102C100020386018401CC00CC00CC00CC00CC00C8C
:102C2000E0086018701038200FC00E172E10010039
:102C30000070007000E001C001800300020000008D
:102C400007C0187020386018401CC00CC00CC00CA5
:102C5000C00CC00CE0086018701038200FC00E17B0
:102C60002E1001000380038007C00EC00C601830D6
:102C70003010000007C0187020386018401CC00CCD
:102C8000C00CC00CC00CC00CE008601870103820DC
:102C90000FC00E152A1001000E081F9011E0200031
:102CA0000000000007C0187020386018401CC00CDD
:102CB000C00CC00CC00CC00CE008601870103820AC
:102CC0000FC00E152A100100183018303870183057
:102CD0000000000007C0187020386018401CC00CAD
:102CE000C00CC00CC00CC00CE0086018701038207C
:102CF0000FC00B0A140D01040600060006000000B8
:102D00000000FFE000000600060006000E10201084
:102D100001FF07CC18782078607840FCC1DCC18CBA
:102D2000C38CC70CC60CEC087C1878107820CFC078
:102D300080000F172E1101001C001C000E00070060
:102D400003000180008000003018F078301830183F
:102D50003018301830183018301830183018301833
:102D6000303818DE0F180F172E1101000070007098
:102D700000E000C001800100020000003018F0787F
:102D80003018301830183018301830183018301803
:102D900030183018303818DE0F180F172E110100B8
:102DA0000380038007C00EE00C6018301010000094
:102DB0003018F078301830183018301830183018B3
:102DC0003018301830183018303818DE0F180F153A
:102DD0002A11010018301C3818301830000000008B
:102DE0003018F07830183018301830183018301883
:102DF0003018301830183018303818DE0F18101FFF
:102E00003E10FFF8001C001C00380070006000C07D
:102E1000008000007E1F1C061C040C0C0E0C0E080B
:102E2000061807180310033003B001A001E001E009
:102E300000C000C000800180018003007E007C0093
:102E4000F8000F20401101F81000F00030003000B1
:102E50003000300030003000300030F03318341CC7
:102E6000380C300E3006300630063006300630049E
:102E7000300C38083C1037E03000300030003000B3
:102E8000300030003000FE00101D3A10FFF8060C34
:102E90000E1C0E1C060C000000007E1F1C061C04ED
:102EA0000C0C0E0C0E08061807180310033003B0A4
:102EB00001A001E001E000C000C0008001800180AD
:102EC00003007E007C00F800000000080002010002
:102ED00000030407000000000000000001020408D5
:102EE0001020408001020408102001020408102074
:102EF00004040404040404040202020202020303A0
:102F00000303030300000000230026002900000043
:102F10000000250028002B000000000024002700EE
:102F20002A004E414E494E495459494E46CDCCCCCB
:102F30003D0AD7233C17B7D13877CC2B329595E68D
:102F4000241FB14F0A000020410000C84200401C6D
:102F50004620BCBE4CCA1B0E5AAEC59D74003D1B1C
:102F6000D22C11241FBECFEFD8E0DEBFCDBF12E0C0
:102F7000A0E0B1E0ECECF8E602C005900D92AC32B6
:102F8000B107D9F725E0ACE2B2E001C01D92A23250
:102F9000B207E1F71FE2C2E6DFE204C02297FE01BA
:102FA0000E94E731CE35D107C9F70E94162D0C9447
:102FB00064340C940000CF93DF93EC01262F4CADCA
:102FC0006BAD04960E948B262BAD992787FD9095BB
:102FD000820F911D8BAF81E090E0DF91CF9108953A
:102FE00060E082E00E94CF2A26E040E855E260E0FF
:102FF00070E083E894E00E94142C40E855E260E021
:1030000070E08EE692E00E94351C80913F0288328B
:1030100011F46FEF03C0823031F463E084E392E097
:103020000E9490280DC0813011F461E0F7CF803309
:1030300039F42FEF4FEF6FEF84E392E00E94932873
:1030400080916D02811107C081E080936D0284E35D
:1030500092E00E943C2884E392E00E946B286AEA96
:1030600070E084E392E00E9430272EE031E04CE0F3
:1030700063E284E392E00E94AB262AE131E04BE177
:1030800064E184E392E00E94AB262DE231E04FE25E
:1030900069E184E392E00E94AB262CE331E04EE349
:1030A0006AE084E392E00E94AB2684E392E00E940F
:1030B00070288111D4CF60ED77E080E090E00C942F
:1030C000432A69E27BE084E392E00E9430278AE0B1
:1030D00080936B028AE280936C0282E00E94082B4C
:1030E00020916E02892BA1F4273030F468E571E05D
:1030F00080E392E00E94632D60916E0270E06D5F4C
:103100007F4F4AE050E080E392E00E940F2E10C013
:103110002A3030F468E571E080E392E00E94632D8C
:103120004AE050E060916E0280E392E00E94242E1B
:1031300064E571E080E392E00E94632D80916F026C
:103140008A3030F468E571E080E392E00E94632DFC
:103150004AE050E060916F0280E392E00E94242EEA
:1031600064E571E080E392E00E94632D809170023B
:103170008A3030F468E571E080E392E00E94632DCC
:103180004AE050E06091700280E392E00E94242EB9
:103190006CE571E080E392E00C94632D6AEA70E0E4
:1031A00084E392E00E94302710926B0280E48093C7
:1031B0006C024AE050E06091730280E392E00E946A
:1031C000242E6DE280E392E00E94652D4AE050E0FB
:1031D0006091720280E392E00E94242E66E571E025
:1031E00080E392E00E94632D4AE050E0609171021A
:1031F00080E392E00C94242E6AEA70E084E392E08B
:103200000E94302710926B028AE080936C024091FA
:10321000860250918702609188027091890222E0B3
:1032200030E080E392E00E94162F6091A60280E3D6
:1032300092E00E94652D6AE571E080E392E00E94D1
:10324000632D40918A0250918B0260918C027091A3
:103250008D0222E030E080E392E00E94162F609120
:10326000A70280E392E00C94652D4F925F926F92DB
:103270007F928F929F92AF92BF92CF92DF92EF9206
:10328000FF92CF93DF93CDB7DEB7AA970FB6F8942E
:10329000DEBF0FBECDBF20E034E244E759E46091C9
:1032A0008A0270918B0280918C0290918D020E9413
:1032B0002D314B015C0120E034E244E759E4609198
:1032C00086027091870280918802909189020E9403
:1032D0002D316B017C018BE1EEE5F1E0DE01119611
:1032E00001900D928A95E1F78BE0E9E7F1E0DE01CC
:1032F0005C9601900D928A95E1F78091A702853442
:1033000049F420E539EA4BE25DE4C501B4010E94CD
:103310001A2F0AC0873551F4A501940160E579EAB6
:103320008BE29DE40E94192F4B015C018091A60263
:103330008E3449F420E539EA4BEA5CE4C701B60172
:103340000E941A2F0AC0833551F4A701960160E547
:1033500079EA8BEA9CE40E94192F6B017C016AEAEE
:1033600070E084E392E00E94302786E580936B0250
:103370008AE080936C0220E836E948E95BE4C50105
:10338000B4010E94822F0E94EA2F2B013C01E1E050
:10339000F0E0EC0FFD1FE60FF71F608180E392E085
:1033A0000E94652D20E836E948E15BE4C701B601DB
:1033B0000E94822F0E94EA2F6FA378A789A79AA75D
:1033C000E1E0F0E0EC0FFD1F8FA198A5E80FF91FD9
:1033D000608180E392E00E94652DD20120E03DE211
:1033E00041E351E00E94F6310E941D309B01AC0187
:1033F000C501B4010E94192F20E030E040E251E401
:103400000E942D3120E030E040EA51E40E94822FFA
:1034100020E034E244E759E40E94822F0E94EA2F20
:10342000ECE1F0E0EC0FFD1FE60FF71F608180E399
:1034300092E00E94652DAFA1B8A520E836E948E9E1
:1034400050E00E94F6310E941D309B01AC01C70183
:10345000B6010E94192F20E034E244E759E40E94AB
:10346000822F0E94EA2FECE1F0E0EC0FFD1FE60F47
:10347000F71F608180E392E00E94652D20E034E236
:1034800044EF59E4C501B4010E94822F4B015C0155
:103490000E94EA2F882777FD8095982F0E941D3083
:1034A0009B01AC01C501B4010E94192F20E030E05E
:1034B00040EC51E40E942D310E94EA2FE1E0F0E05F
:1034C000EC0FFD1FE60FF71F608180E392E00E9482
:1034D000652D20E034E244E759E4C701B6010E94BB
:1034E000822F6B017C010E94EA2F882777FD80954F
:1034F000982F0E941D309B01AC01C701B6010E94AC
:10350000192F20E030E040EC51E40E942D310E9460
:10351000EA2FE1E0F0E0EC0FFD1FE60FF71F6081FE
:1035200080E392E0AA960FB6F894DEBF0FBECDBF3F
:10353000DF91CF91FF90EF90DF90CF90BF90AF9051
:103540009F908F907F906F905F904F900C94652D1F
:103550006AEA70E084E392E00E94302780E580937D
:103560006B0280E480936C028091AB02843178F42A
:1035700064E871E080E392E00E94632D6091AB0209
:1035800070E04AE050E080E392E00C940F2E089542
:10359000CF92DF92EF92FF928EE692E00E94661B3E
:1035A0008EE692E00E944F1C81111AC0C0902C023E
:1035B000D0902D02E0902E02F0902F020E94142A4B
:1035C0006C157D058E059F05B8F40E94142A609342
:1035D0002C0270932D0280932E0290932F020CC028
:1035E0008EE692E00E94521CBC018EE692E00E94A0
:1035F000681C8111DBCF3CC00E94142AC0902C02B1
:10360000D0902D02E0902E02F0902F026C197D09CF
:103610008E099F09693E73408105910548F10E941A
:10362000142A60932C0270932D0280932E029093A3
:103630002F0280916D02811107C081E080936D029D
:1036400084E392E00E943C2884E392E00E946B288D
:103650000E9461180E94CE180E94FC180E94A81AAD
:103660000E94351984E392E00E9470288111F0CF06
:10367000FF90EF90DF90CF900895CF93DF9363E8B2
:1036800074E08EE692E00E94241C109233021092A5
:103690003202C0E3D2E08FE891E09983888342E070
:1036A00060E071E0CE010E94022387E991E09983F6
:1036B00088830E94142A60932C0270932D028093B9
:1036C0002E0290932F02DF91CF910895CF93DF9335
:1036D000FC01E65BFF4F2081222311F080E065C0F2
:1036E000EC01C55BDF4FA881B981109741F0ED91E6
:1036F000FC9111970480F581E02DCD010BC0EC0108
:10370000C35BDF4F88819981DC01ED91FC910480DE
:10371000F581E02D0995892B09F388819981DC01D8
:10372000ED91FC910680F781E02D09958A3049F5ED
:103730009091C202E091C002F091C102E90FF11D27
:1037400010822091C0023091C102B3E02B333B07BD
:1037500039F443EC52E05093C1024093C00208C0D8
:103760002BE333E03093C1022093C00223EC32E01C
:103770003093BF022093BE021092C20291E0909358
:10378000BD02E091C002F091C1029091C20221E01D
:10379000290F2093C202E90FF11D80839091C2028C
:1037A000983718F097E79093C202DF91CF91089570
:1037B000FC01DC01A55BBF4F11961C921E92129674
:1037C00011961C921E921092BD0213971C92109299
:1037D000C2028BE393E09093C1028093C00283EC1A
:1037E00092E09093BF028093BE0215AE14AE158294
:1037F0001482138212821182108212AE11AE10AEA8
:1038000013AE1782168214AA15AA16AA17AA10AA0E
:1038100011AA12AA13AA14A615A616A617A610A6D0
:1038200011A612A613A614A215A216A217A210A2E0
:1038300011A212A213A21486158616861786108668
:1038400011861286138608950F931F93CF93DF93EB
:10385000EC018B010E94D81BC35BDF4F19830883E7
:10386000DF91CF911F910F910895FC01E55BFF4F10
:10387000208131812115310521F0C9010E94742276
:1038800008C0FC01E35BFF4F26E0808191810E942C
:10389000142C6AE070E080E090E00C94432A809160
:1038A000BD0208951092BD028091BE029091BF02A8
:1038B000089560335CF06A3314F480ED05C08FEB3B
:1038C000860F863018F489EC860F089580E00895FD
:1038D0002F923F924F925F926F927F928F929F9220
:1038E000AF92BF92CF92DF92EF92FF920F931F930E
:1038F000CF93DF93CDB7DEB72A970FB6F894DEBF2C
:103900000FBECDBF8C017B01FB0101900020E9F7C8
:103910003197E61BF70B6F0124E0C21AD108DB01D7
:10392000AC0DBD1D8C918A3261F55B01AE0EBF1EE0
:10393000F50133976081C8010E94591C30E1839FD3
:1039400030011124F50132976081C8010E94591C91
:10395000D301A80FB11DCD0142E0242F30E02C157A
:103960003D0558F4F701E20FF31F2081332727FDAF
:103970003095822793274F5FF0CF892B11F080E09D
:10398000E1C46BE971E0C7010E947032892B09F430
:1039900068C26CE270E0C7010E94563201961C01B9
:1039A0000E940D326B017C010E94EF2F4B015C01E4
:1039B00020E137E240E050E00E94A431F80120838A
:1039C00044E6442E512C612C712CA30192010E94DB
:1039D000A431D80111962C93C501B401A301920121
:1039E0000E94A431F801628320E030E040E85FE308
:1039F000C701B6010E945F3020E030E04AE754E49E
:103A00000E942D310E94EF2FD80117967C936E9360
:103A100016976CE270E0C1010E9456327C015C0195
:103A2000BFEFAB1ABB0AFC0181818C3209F4A5C03F
:103A300042E050E0B501CE0101960E9461321B8246
:103A4000CE0101960E942F329B01AC0160E876E91D
:103A500088E990E00E9494312B013C01B7016D5F31
:103A60007F4F42E050E0CE0101960E946132570143
:103A7000F6E0AF0EB11C44E050E0B501CE01039674
:103A80000E9461321F82CE0101960E942F329B015B
:103A9000AC01A2E3B0E00E94EB3123E030E040E073
:103AA00050E00E94C63169017A01D301C201820F40
:103AB000931FA41FB51FF801808B918BA28BB38B32
:103AC000C301B20120EA36E841E050E00E94C6316D
:103AD000CA01B9010E941D302B013C01C701B6018A
:103AE0000E941D302CE933E549EC56E30E942D314C
:103AF0009B01AC01C301B2010E941A2F6B017C0132
:103B0000D80118966D937D938D939C931B9720E01D
:103B100030E048EC52E40E94822F0E94EA2F2B01F1
:103B20003C0184E6849DB001859D700D1124882799
:103B300077FD8095982F0E941D309B01AC01C70135
:103B4000B6010E94192F20E030E040E752E40E94C5
:103B5000822F6B017C01B201882777FD8095982F19
:103B60000E941D309B01AC01C701B6010E941A2FB3
:103B7000F801608F718F828F938F6CE270E0C501C6
:103B80000E945632FC01019621812C3209F1233525
:103B900071F4D80158964D915D916D917C915B9730
:103BA000705858964D935D936D937C935B972181EC
:103BB0002E3419F4F80120AF0BC0233521F4D801BD
:103BC000D8962C9305C02C3209F0D9CEF80110AE4E
:103BD0006CE270E00E9456327C015C01FFEFAF1A8C
:103BE000BF0ADC0111968C918C3209F4A5C043E028
:103BF00050E0B501CE0101960E9461321C82CE01D7
:103C000001960E942F329B01AC0160E876E988E9B9
:103C100090E00E9494312B013C01B7016C5F7F4F13
:103C200042E050E0CE0101960E9461325701B7E0B8
:103C3000AB0EB11C44E050E0B501CE0103960E94EA
:103C400061321F82CE0101960E942F329B01AC018E
:103C5000A2E3B0E00E94EB3123E030E040E050E02E
:103C60000E94C63169017A01D301C201820F931FFC
:103C7000A41FB51FF801848B958BA68BB78BC3014E
:103C8000B20120EA36E841E050E00E94C631CA01A4
:103C9000B9010E941D302B013C01C701B6010E94F1
:103CA0001D302CE933E549EC56E30E942D319B0190
:103CB000AC01C301B2010E941A2F6B017C01D80133
:103CC0001C966D937D938D939C931F9720E030E01D
:103CD00048EC52E40E94822F0E94EA2F2B013C0103
:103CE00084E6849DB001859D700D1124882777FDA1
:103CF0008095982F0E941D309B01AC01C701B60131
:103D00000E94192F20E030E040E752E40E94822F09
:103D10006B017C01B201882777FD8095982F0E9466
:103D20001D309B01AC01C701B6010E941A2FF8019A
:103D3000648F758F868F978F6CE270E0C5010E944B
:103D40005632FC01019621812C3209F1273571F49C
:103D5000D8015C964D915D916D917C915F97705803
:103D60005C964D935D936D937C935F97218127358E
:103D700019F4F80121AF0BC0253421F4D801D996EC
:103D80002C9305C02C3209F0FACDF80111AE6CE28B
:103D900070E00E9456327C01FFEFEF1AFF0ADC014F
:103DA00011968C918C3229F0C7010E941132F801D2
:103DB00084AF6CE270E0C7010E9456327C01FFEFD5
:103DC000EF1AFF0ADC0111968C918C3229F0C701A1
:103DD0000E941132F80185AF6CE270E0C7010E94C9
:103DE00056327C01FFEFEF1AFF0ADC0111968C912D
:103DF0008C3241F0C7010E940D32F80164AB75AB03
:103E000086AB97AB6CE270E0C7010E9456327C0132
:103E1000FFEFEF1AFF0ADC0111968C918C3241F012
:103E2000C7010E940D32F80164A375A386A397A36E
:103E30006CE270E0C7010E9456326CE270E00196BD
:103E40000E945632DC0111962C912C3209F479C271
:103E500001960E940D32F80160A371A382A393A37F
:103E600070C262EA71E0C7010E947032892B09F4C6
:103E700086CD6CE270E0C7010E94563201961C01AB
:103E80000E940D326B017C010E94EF2F4B015C01FF
:103E900020E137E240E050E00E94A431D8012C93A9
:103EA00034E6432E512C612C712CA30192010E9407
:103EB000A431F8012183C501B401A30192010E943C
:103EC000A431D80112966C9320E030E040E85FE323
:103ED000C701B6010E945F3020E030E04AE754E4B9
:103EE0000E942D310E94EF2FF801778366836CE2E8
:103EF00070E0C1010E945632DC0111962C912134F0
:103F000021F421E0F80123AF06C0263509F037CDB2
:103F1000D801DB961C926CE270E001960E9456324A
:103F20007C015C01BFEFAB1ABB0AFC0181818C32C2
:103F300009F4A5C042E050E0B501CE0101960E940F
:103F400061321B82CE0101960E942F329B01AC018F
:103F500060E876E988E990E00E9494312B013C0109
:103F6000B7016D5F7F4F42E050E0CE0101960E94A5
:103F700061325701F6E0AF0EB11C44E050E0B501EC
:103F8000CE0103960E9461321F82CE0101960E94EB
:103F90002F329B01AC01A2E3B0E00E94EB3123E0A1
:103FA00030E040E050E00E94C63169017A01D3015F
:103FB000C201820F931FA41FB51FF801808B918B44
:103FC000A28BB38BC301B20120EA36E841E050E096
:103FD0000E94C631CA01B9010E941D302B013C016B
:103FE000C701B6010E941D302CE933E549EC56E3C8
:103FF0000E942D319B01AC01C301B2010E941A2F16
:104000006B017C01D80118966D937D938D939C93E1
:104010001B9720E030E048EC52E40E94822F0E947F
:10402000EA2F2B013C0184E6849DB001859D700D33
:104030001124882777FD8095982F0E941D309B01C1
:10404000AC01C701B6010E94192F20E030E040E723
:1040500052E40E94822F6B017C01B201882777FD18
:104060008095982F0E941D309B01AC01C701B601BD
:104070000E941A2FF801608F718F828F938F6CE2EC
:1040800070E0C5010E945632FC01019621812C325C
:1040900009F1233571F4D80158964D915D916D91D8
:1040A0007C915B97705858964D935D936D937C937C
:1040B0005B9721812E3419F4F80120AF0BC0233512
:1040C00021F4D801D8962C9305C02C3209F057CC96
:1040D000F80110AE6CE270E00E9456327C015C0187
:1040E000FFEFAF1ABF0ADC0111968C918C3209F4F4
:1040F000A5C043E050E0B501CE0101960E946132B7
:104100001C82CE0101960E942F329B01AC0160E817
:1041100076E988E990E00E9494312B013C01B701D7
:104120006C5F7F4F42E050E0CE0101960E94613209
:104130005701B7E0AB0EB11C44E050E0B501CE0131
:1041400003960E9461321F82CE0101960E942F3297
:104150009B01AC01A2E3B0E00E94EB3123E030E030
:1041600040E050E00E94C63169017A01D301C201EA
:10417000820F931FA41FB51FF801848B958BA68B0C
:10418000B78BC301B20120EA36E841E050E00E945B
:10419000C631CA01B9010E941D302B013C01C70183
:1041A000B6010E941D302CE933E549EC56E30E942C
:1041B0002D319B01AC01C301B2010E941A2F6B018A
:1041C0007C01D8011C966D937D938D939C931F97D2
:1041D00020E030E048EC52E40E94822F0E94EA2F57
:1041E0002B013C0184E6849DB001859D700D112456
:1041F000882777FD8095982F0E941D309B01AC0188
:10420000C701B6010E94192F20E030E040E752E4D8
:104210000E94822F6B017C01B201882777FD809577
:10422000982F0E941D309B01AC01C701B6010E946E
:104230001A2FF801648F758F868F978F6CE270E06C
:10424000C5010E945632FC01019621812C3209F1F0
:10425000273571F4D8015C964D915D916D917C91FB
:104260005F9770585C964D935D936D937C935F97C9
:104270002181273519F4F80121AF0BC0253421F431
:10428000D801D9962C9305C02C3209F078CBF801CF
:1042900011AE6CE270E00E9456327C01FFEFEF1A23
:1042A000FF0ADC0111968C918C3241F0C7010E940B
:1042B0000D32F80160A771A782A793A76CE270E0A6
:1042C000C7010E9456327C01FFEFEF1AFF0ADC01A2
:1042D00011968C918C3241F0C7010E940D32F80189
:1042E00064A775A786A797A76CE270E0C7010E9434
:1042F0005632DC0111962C912C3219F101960E9454
:104300000D320E94EF2F2B013C0120E137E240E00B
:1043100050E00E94A431F801258324E6C22ED12C5E
:10432000E12CF12CA70196010E94A431D80114962A
:104330002C93C301B201A70196010E94A431F80198
:10434000638381E02A960FB6F894DEBF0FBECDBF1F
:10435000DF91CF911F910F91FF90EF90DF90CF9061
:10436000BF90AF909F908F907F906F905F904F9095
:104370003F902F900895E091F503F091F603E81730
:10438000F90769F4A389B4899C918589809589236B
:104390008C931092F6031092F50381E0089580E06B
:1043A0000895CF93DF93EC018A8D9B8D892BF1F0DB
:1043B0008091F5039091F6038C179D07B9F0009753
:1043C00011F00E94BB218E8D8E7F8E8F1092B403D0
:1043D0001092B303D093F603C093F503EB89FC89E5
:1043E00080819D89892B808381E001C080E0DF91FD
:1043F000CF9108951F920F920FB60F9211242F9311
:104400003F934F935F936F937F938F939F93AF935C
:10441000BF93EF93FF93E091F503F091F60330978C
:1044200009F451C0868DA685B785958581FF04C0A6
:104430008C91892329F447C08C91892309F043C0CA
:10444000A389B4899C918589809589238C938689D9
:1044500097890197F1F7208D318DA685B7857585F0
:1044600058E040E0C9010197F1F7842F90E095955D
:104470008795482F6C91672309F04068515091F758
:10448000868D81FD40958091B40390E001968F73F5
:1044900099272091B303281749F0A091B403B0E005
:1044A000AB54BC4F4C938093B40303C0868D8160A2
:1044B000868F828D938D0197F1F7A389B4898C91B2
:1044C0009589892B8C93FF91EF91BF91AF919F912B
:1044D0008F917F916F915F914F913F912F910F90AD
:1044E0000FBE0F901F901895CF93DF93EC019A01A8
:1044F000AB011B8E1A8E198E188E1F8A1E8A60E8D9
:1045000074E88EE190E00E94C631C9012430310583
:1045100020F0B9016350710902C061E070E07D8F45
:104520006C8FEC85E63108F068C0B9017695679527
:104530006431710518F06351710902C061E070E0E7
:104540007F8B6E8B069718F0C901059702C081E03A
:1045500090E0998F888FC901880F991F820F931F50
:1045600096958795969587958D30910510F00C97C7
:1045700002C081E090E09B8F8A8F20916800E83034
:1045800050F091E0EE3008F490E081E001C0880F37
:104590009A95EAF701C084E0822B809368002C850D
:1045A000283038F02E3040F0263148F48CE690E088
:1045B00008C08DE690E005C08BE690E002C080E088
:1045C00090E09C8B8B8B283030F481E001C0880F09
:1045D0002A95EAF70DC0822F90E02E3010F408974C
:1045E00001C00E9791E001C0990F8A95EAF7892FD3
:1045F0008D8B8C8D9D8D0197F1F7CE01DF91CF9141
:104600000C94D121FC0113AE14AE15AE04960C949B
:104610004E280F93FC010150040F84A996A994170A
:1046200018F0081728F402C0081750F0041740F4D7
:104630002150260F83A995A9961720F4281720F456
:1046400080E007C0281720F481E0261710F0F8CF8B
:1046500081E00F910895DB011496ED91FC9115977F
:1046600020E030E061E00994DB011496ED91FC91CB
:10467000159720E030E063E00994DB011496ED919A
:10468000FC91159720E030E040E064E00994DB0104
:104690001496ED91FC91159720E030E041E064E044
:1046A0000994DB011496ED91FC91159720E030E020
:1046B00062E00994DB011496ED91FC91159720E0DE
:1046C00030E065E00994DB011496ED91FC911597BB
:1046D00066E00994AF92BF92CF92DF92EF92FF9281
:1046E0000F931F93CF93DF931F92CDB7DEB75C017B
:1046F0008B017A0180E0F7014491811109C04F3F9D
:10470000D9F1B801C5010E945A2381112EC039C0C8
:104710004F3FB9F34E3FB9F1403F38F5403E30F0DE
:104720004F70B801C5010E9451231FC0403D30F0B9
:104730004F70B801C5010E94342317C0403CB8F047
:10474000B801C50149830E943D2349814295407FBC
:104750004E5FC42ED12CC6010E94D724B801C501DA
:104760000E944723C6010E94D72480E006C047FD6F
:10477000FCCF842F90E0F7CF81E0FFEFEF1AFF0A24
:10478000BACF80E001C081E00F90DF91CF911F91FF
:104790000F91FF90EF90DF90CF90BF90AF90089572
:1047A000CF93DF93EC018BA5882381F088E70E94EB
:1047B0008324882369F08EA1811106C00E94B4244D
:1047C000882331F01BA602C080E4F8CF81E001C04D
:1047D00080E0DF91CF9108951F93CF93DF93142F43
:1047E000E9016330B9F050F4613079F0623009F0DA
:1047F00043C0FC0146A321E023A73EC0663001F17F
:10480000673059F16530C1F50EC0FC0186A50E94E4
:10481000512432C0FC0116A221E023A741112CC073
:104820000E94D02429C00E94D023811103C00E947D
:10483000D02424C0812F0E94B42481111DC0F7CF41
:104840000E94D023882399F31123B1F089910E940B
:10485000B424882361F31150F7CF0E94D02388231A
:1048600031F3112349F0FE0184910E94B42488237E
:1048700029F021961150F5CF81E001C080E0DF9151
:10488000CF911F9108959091F903911104C08093E5
:10489000F9036093F70308951092F9031092F70358
:1048A00008958093F8031092B90084FF02C082E05B
:1048B00001C080E28093B8000C944C24CF93DF9326
:1048C00000D0CDB7DEB720ED37E03A832983909151
:1048D000BC00982391F429813A81232B49F48091DB
:1048E000F80381FD0AC081E00E94432480E006C0F5
:1048F00029813A8121503109E8CF81E00F900F9052
:10490000DF91CF910895CF93C82F84EA8093BC00A4
:1049100061E080E80E945E24882309F19091B9004B
:10492000987F983021F0903111F061E015C0C0936C
:10493000BB0084E88093BC0062E080E80E945E24B3
:10494000882369F08091F80381FD0BC08091B90044
:10495000887F883131F062E082E00E94432480E069
:1049600001C081E0CF9108958093BB0084E88093DB
:10497000BC0063E080E80E945E24882369F0809197
:10498000F80381FD0BC08091B900887F883231F037
:1049900063E082E00E94432480E0089581E008956E
:1049A00084E98093BC0064E080E10C945E242EECEA
:1049B00037E0009729F0F9013197F1F70197F9CF26
:1049C0000895BF92CF92DF92EF92FF920F931F93C1
:1049D000CF93DF938C01EB01B42E690180E148177E
:1049E000B1F1841770F0EAE04E133CC042E0C80118
:1049F0000E942B2344E850E0BE01C8010E946A23B4
:104A000031C0F1E14F1731F185E148132BC0EA8045
:104A1000FB804CE750E0C8010E946A23F701448103
:104A2000406BBE01C8010E945A2341E0BE01C8018B
:104A30000E945123AE01B801C7010E9408298823B2
:104A400001F140E0BE01C8010E9434230BC043E7DE
:104A500050E002C048E650E0BE01C8010E946A234F
:104A600081E010C096014B2DBE01C801DF91CF91AE
:104A70001F910F91FF90EF90DF90CF90BF900C941B
:104A8000802980E0DF91CF911F910F91FF90EF90EF
:104A9000DF90CF90BF900895FC01E60FF11D849147
:104AA00090E0982F88273196E4918E0F911D0895FC
:104AB000FC01849108950E945825882311F08230CA
:104AC00011F486E0089583E0089580E0089566E09B
:104AD0000C944C2568E00C944C250A96FC018491BA
:104AE00008950B96FC0184910895BF92CF92DF92B6
:104AF000EF92FF920F931F93CF93DF93EC01E62E7B
:104B00000C811D81C8010E945825F82E8C819D8141
:104B10000E945B25B82E21E0F21619F0CC24CA942D
:104B200002C05FE0C52E8C819D810E946D25F82E0C
:104B30008C819D810E947125D82E8C819D810E943F
:104B40006A25E0E6EE1538F4009729F0080F191FE2
:104B500041E6F42E10C08C819D810E946725F0E40F
:104B6000FE1538F4009729F0080F191F31E4F32ED1
:104B700002C00F5E1F4FDE1440F4188A1B8A1C8A85
:104B8000198A1A8A80E090E050C0DF14B0F32B2D10
:104B900030E0F80184918F3F19F40F5F1F4F40C040
:104BA000FE1036C08C819D810E94582598012F5F90
:104BB0003F4FF801882311F0823091F484918B8B60
:104BC000F90124912C8BF8013396E491E88BF801DC
:104BD0003496E491E98BF8013596E491EA8B16C09E
:104BE0009491892F8F7082508A8B92959F70998BA8
:104BF000F9012491822F8F708C8B22952F702B8B33
:104C0000F8013296E491E295EF70E88BC8010DC08F
:104C1000F8013296E491EC210E0F111D020F131FC3
:104C2000FD1409F4AACFF394B4CFDF91CF911F9173
:104C30000F91FF90EF90DF90CF90BF9008954F922B
:104C40005F927F928F929F92AF92BF92CF92DF92AC
:104C5000EF92FF920F931F93CF93DF931F92CDB7E5
:104C6000DEB72C01162F742E622F0E9475256C0161
:104C7000009709F43EC0F201848195810E945B2572
:104C8000F82EF201838804899188910E8289781A1E
:104C9000172D101B282D412F692DC2010E940923B9
:104CA000882321F1CF0CD11CF7E08F0E86948694D7
:104CB0008694A82CB12C1715C9F0392D76018E2DAC
:104CC0008C19881578F4F701049120E0412F632FA7
:104CD000C20139830E947F28FFEFEF1AFF0A398152
:104CE000385FEDCFCA0CDB1C1F5FE5CFF201808976
:104CF00001C080E00F90DF91CF911F910F91FF9045
:104D0000EF90DF90CF90BF90AF909F908F907F906B
:104D10005F904F9008950F931F93CF93DF9300D030
:104D20001F92CDB7DEB78C01DC015596ED91FC9159
:104D300056972B834A83698309954A81480F2B81B3
:104D40006981C8010F900F900F90DF91CF911F9153
:104D50000F910C941F26AF92BF92DF92EF92FF92B9
:104D60000F931F93CF93DF9300D0CDB7DEB78C01A5
:104D7000E62EF42EDC015596ED91FC915697298391
:104D80003A830995F80E2981A22E3A81B32ED12CAF
:104D9000F50121915F01222341F04F2D6E2DC801B5
:104DA0000E941F26E80ED80EF3CF8D2D0F900F9086
:104DB000DF91CF911F910F91FF90EF90DF90BF9007
:104DC000AF900895DC0114968D919C9115970097F2
:104DD00009F43FC057962C915797FC01211108C048
:104DE0003596E4915896EC935897FC013C9611C087
:104DF000213041F43F96E4915896EC935897FC018A
:104E0000709607C03D96E4915896EC935897FC0134
:104E10003E96849159968C93599758968C915897B1
:104E2000992787FD909559962C915997821B910946
:104E300027FD93955A962C915A97203441F0829FE2
:104E4000C0011124E6E096958795EA95E1F75B9617
:104E50008C93089525E635E2FC01368B258B089569
:104E6000CF93DF93EC018C819D818617970749F0E2
:104E70007D836C83CE010E94E22685E695E29E8BBF
:104E80008D8BDF91CF9108951F93CF93DF93EC012A
:104E90001D821C821F821E82198681E0888782E221
:104EA0008A871F861E8680E090E02FEFFE01E80FC4
:104EB000F91F23A301968E309105C1F711E018A3C5
:104EC000CE010E942A271F8B188E198E80E48A8FAC
:104ED0001B8E89EC99E29AAB89ABDF91CF911F9140
:104EE0000895DB01ED91FC910994EF92FF921F93DD
:104EF000CF93DF9300D0CDB7DEB77C01DC01D19634
:104F0000ED91FC91D29782E069837A83099520E044
:104F100030E04AE069817A81C7010E947127182F29
:104F2000D701D196ED91FC91D29783E00995D701F5
:104F3000D196ED91FC91D29780E00995812F0F9049
:104F40000F90DF91CF911F91FF90EF9008950F93F5
:104F50001F93CF93DF93EC018B01E9A9FAA982E0BB
:104F60000995E9A9FAA981E0099520E030E044E13A
:104F7000B801CE010E9471279E012D5C3F4F47E191
:104F8000B801CE010E947127E9A9FAA980E0DF915A
:104F9000CF911F910F910994FF920F931F93CF937D
:104FA000DF93EC018B01E9A9FAA982E00995E9A94F
:104FB000FAA981E0099520E030E045E1B801CE0191
:104FC0000E947127F82E882341F09E012D5C3F4FEF
:104FD00047E1B801CE010E947127E9A9FAA980E052
:104FE00009958F2DDF91CF911F910F91FF9008951B
:104FF000CF93DF931F92CDB7DEB79E012F5F3F4F58
:1050000046E40E94712789810F90DF91CF91089526
:10501000CF93DF931F92CDB7DEB79E012F5F3F4F37
:1050200047E40E94712789810F90DF91CF91089505
:1050300020E030E048E40C947127CF93DF93EC013B
:105040006A817B810E94F82788836A817B81CE01F7
:105050000E94082889836A817B81CE010E941828DA
:105060008B879E012D5C3F4F6A817B8147E1CE019A
:10507000DF91CF910C947127CF93DF93EC016A817C
:105080007B810E947527882329F0CE010E941D286C
:1050900081E001C080E0DF91CF910895EF92FF920F
:1050A0000F931F93CF93DF931F92CDB7DEB77C0191
:1050B0008B0149830E944427F701138302834981AE
:1050C00046A7C7010F90DF91CF911F910F91FF90DD
:1050D000EF900C943C28FC01628173810C94A7270B
:1050E000CF93DF93EC01EE85FF85309709F00995AA
:1050F0006A817B81CE01DF91CF910C94CC270F93F5
:10510000FC0182819381648F458F278F068F9F01D9
:10511000245E3F4F4BE3BC01CF010F910C947127EC
:10512000FC0160A308954695469530E2439FF00147
:1051300011242695269526952E2BFC0120A3469515
:1051400046954695687F462B41A30895FC0112823F
:1051500080818150838314820895FC0120818281A3
:10516000820F82839181891760F484818F5F8483A9
:105170008381820F891710F08FEF890F838381E07D
:10518000089580E00895DC011696ED91FC91179743
:1051900015968C919F01280F311DC9011192E817B6
:1051A000F907E1F70895FC0191E08381861708F47F
:1051B00090E021E0461708F020E0322F392B81E003
:1051C0005281451708F480E083239223892B0895A8
:1051D000DC01FB01108212968C9112978183159647
:1051E0008C9115978150828313968C9183830895B7
:1051F000FB0141812381213029F0233031F468EF14
:10520000640F04C0642F485F01C0642F0C94D3283E
:10521000FC01CB01BA012681378145810C946323BF
:10522000DC011696ED91FC91179712968C91481B14
:10523000477081E090E0042E01C0880F0A94EAF7DD
:10524000E60FF11D3081222311F0832B02C08095DF
:10525000832380830895FB014181DC0112962C9108
:105260001297421768F013962C911397241740F069
:10527000608115962C91621718F424810C941029E2
:105280000895CF92DF92FF920F931F93CF93DF93F6
:1052900000D0CDB7DEB78C016B01FB01F2808381BA
:1052A000813039F070F0823039F0833041F020E005
:1052B00001C021E030E007C020E03FEF04C02FEF45
:1052C000F9CF20E031E0F7FE08C0B601C80129831C
:1052D0003A830E942B293A812981F6018081830F2C
:1052E00080838181820F8183FF0C69F70F900F907B
:1052F000DF91CF911F910F91FF90DF90CF90089594
:105300000F931F93CF93DF938901FB01C281D38158
:105310004233F9F068F4453109F1473141F1443144
:1053200081F5CE010E94C328CE010E94A62829C083
:10533000463411F1473411F14B3319F5B901CE015F
:105340000E94F8288823E9F0B801CE010E94412983
:1053500018C0B901CE010E942B2913C0CE010E94B2
:10536000AD28882381F0CE010E94C3280AC0B9016C
:10537000CE010E94E82805C08D8101C08981F80115
:10538000808381E001C080E0DF91CF911F910F9178
:10539000089508951F920F920FB60F9211242F9324
:1053A0003F938F939F93AF93BF9380917B04909192
:1053B0007C04A0917D04B0917E0430917A0426E0B3
:1053C000230F2D3720F40296A11DB11D05C029E839
:1053D000230F0396A11DB11D20937A0480937B04B3
:1053E00090937C04A0937D04B0937E0480917F040D
:1053F00090918004A0918104B09182040196A11D36
:10540000B11D80937F0490938004A0938104B09396
:105410008204BF91AF919F918F913F912F910F90F7
:105420000FBE0F901F9018952FB7F89460917B04D2
:1054300070917C0480917D0490917E042FBF08952B
:105440003FB7F89480917F0490918004A0918104EB
:10545000B091820426B5A89B05C02F3F19F0019694
:10546000A11DB11D3FBF6627782F892F9A2F620F8C
:10547000711D811D911D43E0660F771F881F991FC5
:105480004A95D1F70895CF92DF92EF92FF92CF9392
:10549000DF936B017C010E94202AEB01C114D1042F
:1054A000E104F10489F00E94182F0E94202A6C1B4D
:1054B0007D0B683E734090F381E0C81AD108E10883
:1054C000F108C851DC4FEACFDF91CF91FF90EF9008
:1054D000DF90CF900895789484B5826084BD84B5C0
:1054E000816084BD85B5826085BD85B5816085BDDF
:1054F000EEE6F0E0808181608083E1E8F0E01082F8
:10550000808182608083808181608083E0E8F0E038
:10551000808181608083E1EBF0E080818460808322
:10552000E0EBF0E0808181608083EAE7F0E0808159
:105530008460808380818260808380818E7F80838D
:105540008081806880831092C1000895833081F04B
:1055500028F4813099F08230A1F008958730A9F0C5
:105560008830B9F08430D1F4809180008F7D03C001
:10557000809180008F7780938000089584B58F7725
:1055800002C084B58F7D84BD08958091B0008F776F
:1055900003C08091B0008F7D8093B0000895CF93B9
:1055A000DF9390E0FC01E452F14D2491FC01E051C5
:1055B000F14D8491882349F190E0880F991FFC01F7
:1055C000E85EF04DA591B491825F904DFC01C591CC
:1055D000D4919FB7611108C0F8948C9120958223D3
:1055E0008C93888182230AC0623051F4F8948C91A4
:1055F000322F309583238C938881822B888304C03B
:10560000F8948C91822B8C939FBFDF91CF9108955A
:10561000CF93DF93282F30E0F901E853F14D8491C7
:10562000F901E452F14DD491F901E051F14DC491E9
:10563000CC2391F081110E94A62AEC2FF0E0EE0F0E
:10564000FF1FEC5FF04DA591B4912C912D2381E0CB
:1056500090E021F480E002C080E090E0DF91CF9103
:105660000895FC01818D228D90E0805C9F4F821B0C
:1056700091098F7399270895FC01918D828D981758
:1056800031F0828DE80FF11D858D90E008958FEF48
:105690009FEF0895FC01918D828D981761F0828DA6
:1056A000DF01A80FB11D5D968C91928D9F5F9F7356
:1056B000928F90E008958FEF9FEF089588EC9CE221
:1056C000892B49F080E090E0892B29F00E94C82CBA
:1056D00081110C9400000895FC01848DDF01A80F56
:1056E000B11DA35ABF4F2C91848D90E001968F730A
:1056F0009927848FA689B7892C93A089B1898C9129
:1057000080648C93938D848D981306C00288F389EE
:10571000E02D80818F7D80830895CF93DF93EC010E
:10572000888D8823C9F0EA89FB89808185FD05C0C1
:10573000A889B9898C9186FD0FC00FB607FCF5CFFB
:10574000808185FFF2CFA889B9898C9185FFEDCF43
:10575000CE010E946C2BE7CFDF91CF910895CF92BD
:10576000DF92FF920F931F93CF93DF931F92CDB7DA
:10577000DEB76C0181E0D60158968C9358975B9602
:105780009C915B975C968C915C97981307C05096A0
:10579000ED91FC915197808185FD2EC0F601038D1E
:1057A00010E00F5F1F4F0F731127F02EF601848D4D
:1057B000F81211C00FB607FCF9CFD6015096ED9143
:1057C000FC915197808185FFF1CFC60169830E94CA
:1057D0006C2B6981EBCF838DE80FF11DE35AFF4FEE
:1057E0006083D6015B960C935B975296ED91FC918A
:1057F0005397808180620CC0D6015696ED91FC9142
:10580000579760835096ED91FC9151978081806409
:10581000808381E090E00F90DF91CF911F910F91F5
:10582000FF90DF90CF900895BF92CF92DF92EF92DA
:10583000FF92CF93DF93EC016A017B01B22E60E807
:1058400074E88EE190E0A70196010E94A4312150F6
:105850003109410951095695479537952795E889AA
:10586000F98982E08083211580E1380798F0E88982
:10587000F989108260E472E48FE090E0A70196015C
:105880000E94A4312150310941095109569547958B
:1058900037952795EC85FD853083EE85FF85208340
:1058A000188EEC89FD89B082EA89FB89808180614C
:1058B0008083EA89FB89808188608083EA89FB890B
:1058C000808180688083EA89FB8980818F7D8083E5
:1058D000DF91CF91FF90EF90DF90CF90BF90089530
:1058E0001F920F920FB60F9211242F938F939F93B5
:1058F000EF93FF93E0919304F09194048081E09101
:105900009904F0919A0482FD12C0908180919C04C8
:105910008F5F8F7320919D04821751F0E0919C045A
:10592000F0E0ED57FB4F958F80939C0401C0808180
:10593000FF91EF919F918F912F910F900FBE0F903C
:105940001F9018951F920F920FB60F9211242F934C
:105950003F934F935F936F937F938F939F93AF93F7
:10596000BF93EF93FF9383E894E00E946C2BFF9129
:10597000EF91BF91AF919F918F917F916F915F91C7
:105980004F913F912F910F900FBE0F901F90189540
:1059900083E894E00E94312B21E0892B09F420E078
:1059A000822F0895109286041092850488EE93E069
:1059B000A0E0B0E08093870490938804A0938904CA
:1059C000B0938A048EE092E09093840480938304E1
:1059D00085EC90E09093900480938F0484EC90E0A9
:1059E000909392048093910480EC90E090939404BF
:1059F0008093930481EC90E09093960480939504B7
:105A000082EC90E0909398048093970486EC90E069
:105A100090939A048093990410929C0410929D0490
:105A200010929E0410929F04089508950E946B2A7C
:105A30000E94152D0E94F017CEE5DBE20E94C81AE5
:105A40002097E1F30E945E2BF9CFCF92DF92EF9285
:105A5000FF920F931F93CF93DF936C017A01EB01B9
:105A6000E60EF71E00E010E0CE15DF0561F069914B
:105A7000D601ED91FC910190F081E02DC6010995D0
:105A8000080F191FF1CFC801DF91CF911F910F911E
:105A9000FF90EF90DF90CF9008956115710581F030
:105AA000DB010D900020E9F7AD0141505109461B83
:105AB000570BDC01ED91FC910280F381E02D0994FC
:105AC00080E090E008950C944D2DDC01ED91FC9167
:105AD0000190F081E02D09948F929F92AF92BF9236
:105AE000CF92DF92EF92FF920F931F93CF93DF93AA
:105AF000CDB7DEB7A1970FB6F894DEBF0FBECDBF0E
:105B00007C01C42EE52FCB01D22E19A221E02D1548
:105B100010F02AE0D22E8E010F5D1F4F8D2C912C9C
:105B2000A12CB12C6C2D7E2FA50194010E94A431D3
:105B30008C2DD29E80191124015011098A3014F441
:105B4000805D01C0895CF801808321153105410524
:105B5000510521F0C22EE32FCA01E4CFB801C701DD
:105B60000E944D2DA1960FB6F894DEBF0FBECDBF9B
:105B7000DF91CF911F910F91FF90EF90DF90CF9029
:105B8000BF90AF909F908F900895CF92DF92EF9249
:105B9000FF920F931F93CF93DF93EC016A017B0178
:105BA0002115310579F4E881F9810190F081E02D2A
:105BB000642FDF91CF911F910F91FF90EF90DF90B5
:105BC000CF9009942A303105E9F477FF1AC06DE2CD
:105BD0000E94652D8C0144275527BA014C195D0997
:105BE0006E097F092AE0CE010E946C2D800F911F63
:105BF000DF91CF911F910F91FF90EF90DF90CF90A9
:105C000008952AE0B701A601CE01DF91CF911F913F
:105C10000F91FF90EF90DF90CF900C946C2D9A0134
:105C2000AB01662757FD6095762F0C94C52D211585
:105C3000310541F4DC01ED91FC910190F081E02D02
:105C4000642F09940C946C2D9A01462F50E060E06B
:105C500070E00C94172E4F925F926F927F928F920A
:105C60009F92AF92BF92CF92DF92EF92FF920F93EB
:105C70001F93CF93DF93EC016A017B01B22E9A014F
:105C8000AB01C701B6010E949031882319F06DE184
:105C900072E027C026013701E89477F82FEF3FEF35
:105CA0004FE75FE7C301B2010E94903181110DC03F
:105CB0002FEF3FEF4FE75FE7C301B2010E947E2F56
:105CC00018161CF461E272E00CC02FEF3FEF4FE7B3
:105CD0005FE4C701B6010E9429311816ACF465E2F1
:105CE00072E0CE01DF91CF911F910F91FF90EF9065
:105CF000DF90CF90BF90AF909F908F907F906F90EC
:105D00005F904F900C944D2D2FEF3FEF4FE75FECDE
:105D1000C701B6010E947E2F87FDE1CF20E030E071
:105D2000A901C701B6010E947E2F87FF0AC06DE25C
:105D3000CE010E94652D8C01F7FAF094F7F8F094EB
:105D400002C000E010E0A12C60E070E080E09FE382
:105D5000AB1441F020E030E040E251E40E94822F99
:105D6000A394F6CF9B01AC01C701B6010E941A2F84
:105D70006B017C010E94EF2F2B013C010E941B3024
:105D80009B01AC01C701B6010E94192F6B017C0178
:105D90002AE0B301A201CE010E946C2D080F191F49
:105DA000BB2039F069E272E0CE010E944D2D080F50
:105DB000191F7B2C772041F120E030E040E251E4D4
:105DC000C701B6010E942D316B017C010E94EA2FB0
:105DD0004B01AA2497FCA094BA2C2AE030E0B5012C
:105DE000A401CE010E94C52D080F191FC501B401E1
:105DF0000E941D309B01AC01C701B6010E94192F02
:105E00006B017C017A94D6CFC801DF91CF911F91AD
:105E10000F91FF90EF90DF90CF90BF90AF909F9049
:105E20008F907F906F905F904F9008950C942B2EE1
:105E300008955058BB27AA270ED0D1C1C2D130F047
:105E4000C7D120F031F49F3F11F41EF4B7C10EF416
:105E5000E095E7FB9FC1E92FD3D180F3BA17620722
:105E600073078407950718F071F49EF5EBC10EF4E3
:105E7000E0950B2EBA2FA02D0B01B90190010C015A
:105E8000CA01A0011124FF27591B99F0593F50F472
:105E9000503E68F11A16F040A22F232F342F4427CA
:105EA000585FF3CF469537952795A795F0405395C2
:105EB000C9F77EF41F16BA0B620B730B840BBAF092
:105EC0009150A1F0FF0FBB1F661F771F881FC2F7FD
:105ED0000EC0BA0F621F731F841F48F48795779511
:105EE0006795B795F7959E3F08F0B3CF9395880FC8
:105EF00008F09927EE0F97958795089527D108F414
:105F000081E008950CD06BC163D140F05AD130F0DC
:105F100021F45F3F19F03EC1511195C14FC170D1BD
:105F200098F39923C9F35523B1F3951B550BBB2760
:105F3000AA2762177307840738F09F5F5F4F220F0D
:105F4000331F441FAA1FA9F333D00E2E3AF0E0E806
:105F500030D091505040E695001CCAF729D0FE2F52
:105F600027D0660F771F881FBB1F261737074807E4
:105F7000AB07B0E809F0BB0B802DBF01FF2793589A
:105F80005F4F2AF09E3F510568F004C15CC15F3F3E
:105F9000ECF3983EDCF3869577956795B795F79582
:105FA0009F5FC9F7880F911D9695879597F908957A
:105FB000E1E0660F771F881FBB1F62177307840716
:105FC000BA0720F0621B730B840BBA0BEE1F88F725
:105FD000E095089504D06894B11135C1089518D1A1
:105FE00088F09F5790F0B92F9927B751A0F0D1F0C2
:105FF000660F771F881F991F1AF0BA95C9F712C04C
:10600000B13081F01FD1B1E008951CC1672F782F06
:106010008827B85F39F0B93FCCF3869577956795B7
:10602000B395D9F73EF490958095709561957F4F23
:106030008F4F9F4F0895E89409C097FB3EF49095C9
:106040008095709561957F4F8F4F9F4F9923A9F051
:10605000F92F96E9BB279395F695879577956795E0
:10606000B795F111F8CFFAF4BB0F11F460FF1BC024
:106070006F5F7F4F8F4F9F4F16C0882311F096E9B7
:1060800011C0772321F09EE8872F762F05C0662365
:1060900071F096E8862F70E060E02AF09A95660F1E
:1060A000771F881FDAF7880F9695879597F90895D7
:1060B00088D018F011F08CD038F480C0C4C0E92F1B
:1060C0009FD0B0F35523C9F3E7FB6217730784072A
:1060D0009507A8F199F3E92FFF2788232AF0319734
:1060E000660F771F881FDAF7952F5527442332F064
:1060F00091505040220F331F441FD2F7BB27E91B9A
:10610000F50B621B730B840BB109C1F222F4620F11
:10611000731F841FB11D31972AF0660F771F881FE8
:10612000BB1FEFCF915050405AF041F0882332F01E
:10613000660F771F881F91505040C1F7939530C06C
:106140008695779567959F5FD9F7F8CF990F0008E7
:10615000550FAA0BE0E8FEEF16161706E807F90739
:10616000C0F012161306E407F50798F0621B730BD4
:10617000840B950B39F40A2661F0232B242B252B55
:1061800021F408950A2609F4A140A6958FEF811DF8
:10619000811D089597F99F6780E870E060E0089599
:1061A0009F3F31F0915020F4879577956795B7958B
:1061B000880F911D9695879597F908959FEF80EC2C
:1061C000089500240A94161617061806090608955D
:1061D00000240A9412161306140605060895092EC3
:1061E0000394000C11F4882352F0BB0F40F4BF2B32
:1061F00011F460FF04C06F5F7F4F8F4F9F4F089572
:1062000057FD9058440F551F59F05F3F71F0479567
:10621000880F97FB991F61F09F3F79F0879508954C
:10622000121613061406551FF2CF4695F1DF08C06B
:10623000161617061806991FF1CF86957105610588
:1062400008940895E894BB2766277727CB0197F930
:1062500008957CDF08F48FEF08950BD0C0CFB1DF35
:1062600028F0B6DF18F0952309F094CFA7CF1124BA
:10627000EACFC6DFA0F3959FD1F3950F50E0551FED
:10628000629FF001729FBB27F00DB11D639FAA278B
:10629000F00DB11DAA1F649F6627B00DA11D661FDA
:1062A000829F2227B00DA11D621F739FB00DA11DFB
:1062B000621F839FA00D611D221F749F3327A00DB5
:1062C000611D231F849F600D211D822F762F6A2F51
:1062D00011249F5750408AF0E1F088234AF0EE0FD6
:1062E000FF1FBB1F661F771F881F91505040A9F7E3
:1062F0009E3F510570F04ECFA6CF5F3FECF3983E26
:10630000DCF3869577956795B795F795E7959F5F49
:10631000C1F7FE2B880F911D9695879597F90895E3
:1063200015DF880B990B0895DB018F939F930E94D3
:10633000EB31BF91AF91A29F800D911DA39F900D56
:10634000B29F900D11240895A1E21A2EAA1BBB1B27
:10635000FD010DC0AA1FBB1FEE1FFF1FA217B30731
:10636000E407F50720F0A21BB30BE40BF50B661F47
:10637000771F881F991F1A9469F76095709580950B
:1063800090959B01AC01BD01CF010895052E97FBAF
:106390001EF400940E94DD3157FD07D00E94A43105
:1063A00007FC03D04EF40C94DD31509540953095A8
:1063B00021953F4F4F4F5F4F089590958095709571
:1063C00061957F4F8F4F9F4F0895EE0FFF1F0590F0
:1063D000F491E02D09940E94FE31A59F900DB49F89
:1063E000900DA49F800D911D11240895B7FF0C946A
:1063F000EB310E94EB31821B930B0895A29FB001F9
:10640000B39FC001A39F700D811D1124911DB29FE8
:10641000700D811D1124911D0895662777270C9416
:10642000A732FC0188279927E89421912032E9F3CB
:10643000293010F02E30C8F32B3241F02D3239F4D0
:10644000689404C00E949F32820F911D21912053B5
:106450002A30C0F31EF4909581959F4F08951F93A5
:10646000FC0199278827BC01E89411911032E9F3C7
:10647000193010F01E30C8F31B3251F01D3249F4B0
:10648000689406C00E948A32610F711D811D911DA2
:10649000119110531A30B0F33EF490958095709599
:1064A00061957F4F8F4F9F4F1F910895FC01819100
:1064B000861721F08823D9F7992708953197CF01BE
:1064C0000895FB01DC014150504048F001900D92CD
:1064D0000020C9F701C01D9241505040E0F70895D7
:1064E000FB0151915523A9F0BF01DC014D914517E6
:1064F0004111E1F759F4CD010190002049F04D918F
:1065000040154111C9F3FB014111EFCF81E090E04B
:1065100001970895592F482F372F262F660F771F81
:10652000881F991F660F771F881F991F620F731F9F
:10653000841F951F660F771F881F991F08957AE0A3
:10654000979F902D879F802D910D11240895A0E095
:10655000B0E0EDEAF2E30C9433348B016115710580
:1065600021F0DB018C9311969C93EC015E01BFEF4F
:10657000AB1ABB0A7501C8808C2D90E00E940D34C7
:10658000892B11F0E501F2CFEDE2CE1208C07E01B9
:10659000F2E0EF0EF11CC980DD24D39409C02BE298
:1065A000C21205C07E0142E0E40EF11CC980D12C6C
:1065B000E701219743E050E06AE27FE2CE010E94CA
:1065C0001534892BC1F4239645E050E065E27FE263
:1065D000CE010E941534892B09F425960115110569
:1065E00019F0D801CD93DC93D11006C160E070E0C2
:1065F00080E89FE70AC143E050E062E27FE2CE011B
:106600000E941534892B59F40115110509F4F9C0BC
:10661000B2E0EB0EF11CF801F182E082F2C0F7016A
:1066200060E070E0CB01C0E0D0E07F01A0EDAA2ED9
:10663000AC0C29E02A1530F14D2D4260B42E2D2DE1
:106640002870D2FE04C0211125C0219623C021113B
:106650002197A5E0B0E09B01AC010E94EB31660FF1
:10666000771F881F991F6A0D711D811D911D683943
:10667000A9E97A078A07A9E19A0760F0BD2DB660FB
:10668000BB2E08C02EEFA2120AC0D3FC50C04D2D65
:106690004860B42E3196D701CC90DB2CC6CF2C2D80
:1066A0002F7D253409F043C0A081AD3241F4BD2DCA
:1066B000B061DB2E7F0122E0E20EF11C0CC07F01F5
:1066C000AB3231F04FEFE41AF40A21E030E006C0BB
:1066D000A2E0EA0EF11CA18122E030E0A053AA3032
:1066E00018F0E21AF30A23C0F70120E030E0203866
:1066F000BCE03B075CF4A901440F551F440F551F34
:10670000240F351F220F331F2A0F311DAF014F5F9A
:106710005F4F7A01A081A053AA3010F4FA01E7CFAD
:10672000D4FE03C0319521953109C20FD31FD1FE8C
:1067300009C00115110531F0E1E0EE1AF108D801A8
:10674000ED92FC920E941B302D2D2370233019F006
:106750004B015C0106C04B015C01B7FAB094B7F87D
:10676000B09420E030E0A901C501B4010E947E2F61
:10677000882309F43EC0D7FF06C0D195C195D10941
:1067800001E41FE202C009E51FE26801B8E1CB1A8B
:10679000D10890E2E92EF12CCE15DF0574F0F80156
:1067A0002591359145915491C501B4010E942D3137
:1067B0004B015C01CE19DF09EFCF04501109F594AC
:1067C000E7940C151D0541F78A2D880F8B2D881F26
:1067D0008F3F49F020E030E0A901C501B4010E94DB
:1067E0007E2F811106C082E290E090932105809374
:1067F0002005C501B40109C060E070E080E89FEFAA
:1068000004C060E070E080EC9FE7CDB7DEB7ECE05D
:106810000C944F349927882708959111FBCF80322B
:1068200019F089508550D0F70895FB01DC014150E3
:10683000504088F08D9181341CF08B350CF4805ED3
:10684000659161341CF06B350CF4605E861B611140
:1068500071F3990B0895881BFCCF2F923F924F92B2
:106860005F926F927F928F929F92AF92BF92CF92E0
:10687000DF92EF92FF920F931F93CF93DF93CDB7E9
:10688000DEB7CA1BDB0B0FB6F894DEBF0FBECDBF61
:1068900009942A88398848885F846E847D848C8432
:1068A0009B84AA84B984C884DF80EE80FD800C813B
:1068B0001B81AA81B981CE0FD11D0FB6F894DEBF1E
:0C68C0000FBECDBFED010895F894FFCF8E
:1068CC00E1240601EC23084000000080FA03475045
:1068DC005320446973706C617900536F66747761EF
:1068EC00726520627920504130525745004D6164E9
:1068FC006520627920524133544F58004750535F02
:10690C00446973706C61795F636F725F74696D65F4
:10691C005F7632003A002D323000202D20004142AB
:10692C00434445464748494A4B4C4D4E4F505152B3
:10693C00535455565758595A003031323334353632
:10694C0037383900536174733A200000000000DBC3
:10695C0017252D00000000DB17252D244750474735
:10696C004100244750524D430024504D544B313874
:10697C00352C302A32320024504D544B3030312CCF
:10698C003138352C332A33430024504D544B313895
:10699C00352C312A32330024504D544B3138332AA4
:1069AC0033380024504D544B4C4F470024504D5419
:1069BC004B3136312C302A32380024504D544B3068
:1069CC0031302C3030322A32440000000000AF2B22
:1069DC00252D312B4A2B3C2B8D2B0D0A006E616E15
:0C69EC0000696E66006F7666002E0000E9
:00000001FF
